:020000040000FA
:1000000025007B0A700869086308700872086F0889
:100010006A0865086308740873082E086F08720878
:1000200067082E0875086B08200828086308290847
:1000300020083208300830083908620869086B085F
:1000400065086C086908670868087408760832084B
:100050002E08480845085808310837082F08300886
:1000600039082F0832083008300839081502E20133
:100070004008430846084B08540859086208070816
:1000800032088708000832080708000812088708A5
:100090001208800800080C0801080C0802080C0867
:1000A00004080C0802080008020807081E080008D7
:1000B0000008020807080A0800083C0887080A0820
:1000C00000080008010807080308000801080708DD
:1000D00003080008010807080308000801080708CA
:1000E00003080008010807080308000801080708BA
:1000F000320800080008080C06001F0C020004006B
:10010000E3068C0A66007500700072007400040C2F
:100110003800400C3600CB0A640C32000602E304BF
:1001200066060300BA0966068C0AF202920AF20514
:10013000BA096607AB0AF2067200FD0CD201720022
:100140000307C90AB5023F09950003067500360981
:1001500036003700CB0AF206C90AB2029C0CD20163
:100160000307C90A660074006607B40ABA090602E2
:10017000E30403001A0C3100F002BC0A3803030642
:10018000580518025401F40714022600F102BC0AB3
:100190000008F302980AD6093300000D4306D30A7B
:1001A000D6093400980A17023600CB0A1602B602A6
:0201B00022002B
:021FFE00EB0FE7
:00000001FF
